:100000000C9415170C941F170C941F170C941F17A2
:100010000C941F170C941F170C941F170C941F1788
:100020000C941F170C941F170C941F170C941F1778
:100030000C941F170C941F170C941F170C941F1768
:100040000C941F170C941F170C941F170C941F1758
:100050000C941F170C941F170C941F170C941F1748
:100060000C941F170C941F172119251929192C19E5
:100070003019341921195E00066600011E04001EA5
:100080000A001E0F001E15001E1B001E2100251E4B
:1000900000201E001A1E00141E000E1E00081E0066
:1000A000031E00001E02001E08001E0E001E13008C
:1000B0001E19001E1F001E2500211E001C1E0016FA
:1000C0001E00101E000A1E00051E00001E06001E57
:1000D0005F00056700001E05001E0A001E10001EBE
:1000E00016001E1C001E2100251E001F1E001A1EC9
:1000F00000141E000E1E00081E00031E00001E023B
:10010000001E08001E0E001E13001E19001E1E00F9
:100110001E2400221E001C1E00171E00111E000BB4
:100120001E00051E00001E05001E6000051E0000CA
:100130001E05001E0B001E11001E17001E1C001EB7
:100140002100251E001F1E00191E00131E000E1E7A
:1001500000081E00031E00001E02001E08001E0EE6
:10016000001E13001E18001E1E001E2400221E006A
:100170001C1E00171E00111E000C1E00061E000093
:100180001E05001E6100041E00001E06001E0C005D
:100190001E11001E17001E1C001E2200241E001F20
:1001A0001E00191E00131E000E1E00081E00031E56
:1001B00000001E02001E08001E0D001E13001E1867
:1001C000001E1E001E2300231E001D1E00171E0001
:1001D000121E000C1E00071E00011E04001E6200FD
:1001E000031E01001E07001E0C001E11001E17003A
:1001F0001E1D001E2200241E001E1E00191E0013BC
:100200001E000E1E00081E00031E00001E02001E1F
:1002100008001E0D001E13001E18001E1E001E23C7
:1002200000231E001E1E00181E00121E000D1E00C0
:10023000071E00011E03001E6300031E01001E07AF
:10024000001E0C001E12001E18001E1D001E2300A2
:10025000241E001E1E00181E00131E000E1E000885
:100260001E00031E00001E02001E07001E0D001EC1
:1002700013001E18001E1E001E2300231E001E1E3B
:1002800000181E00131E000D1E00081E00021E0393
:10029000001E6400021E02001E08001E0D001E1338
:1002A000001E18001E1E001E2300231E001E1E001E
:1002B000181E00131E000E1E00081E00031E000064
:1002C0001E02001E07001E0D001E12001E18001E3A
:1002D0001E001E2300231E001E1E00181E00131EDB
:1002E000000E1E00081E00031E02001E6500011EF7
:1002F00003001E08001E0E001E13001E18001E1E06
:10030000001E2300231E001E1E00181E00131E00C8
:100310000E1E00081E00031E00001E02001E070025
:100320001E0D001E12001E18001E1D001E2300249C
:100330001E001E1E00191E00131E000E1E00081EA9
:1003400000031E01001E6600011E03001E08001EA1
:100350000E001E13001E19001E1E001E2300231E69
:10036000001E1E00181E00131E000E1E00081E0098
:10037000031E00001E02001E07001E0D001E1200BC
:100380001E17001E1D001E2200241E001F1E001A24
:100390001E00141E000F1E00091E00041E01001E78
:1003A0006700001E04001E09001E0F001E14001E20
:1003B00019001E1F001E2400231E001D1E00181EF3
:1003C00000131E000D1E00081E00031E00001E026A
:1003D000001E07001E0C001E12001E17001E1C002F
:1003E0001E2200251E001F1E001A1E00151E0010D2
:1003F0001E000A1E00051E00001E1E00001E050035
:100400001E0A001E0F001E15001E1A001E1F001ED1
:100410002400221E001D1E00181E00121E000D1EAC
:1004200000081E00031E00001E02001E07001E0C16
:10043000001E11001E17001E1C001E2100251E009C
:100440001F1E001A1E00151E00101E000A1E0005A9
:100450001E00001E1E00001E05001E0A001E0F00CA
:100460001E15001E1A001E20001E2500221E001D43
:100470001E00171E00121E000D1E00081E00031E87
:1004800000001E02001E07001E0C001E11001E1799
:10049000001E1C001E2100251E00201E001B1E0029
:1004A000151E00101E000B1E00061E00001E1E0161
:1004B000001E06001E0B001E10001E15001E1A0056
:1004C0001E20001E2500211E001C1E00171E0012EB
:1004D0001E000D1E00081E00031E00001E02001E4E
:1004E00007001E0C001E11001E17001E1C001E21FE
:1004F00000251E00201E001B1E00161E00111E00DF
:100500000C1E00071E00011E1E01001E07001E0C0F
:10051000001E11001E16001E1B001E20001E2500BE
:10052000211E001C1E00171E00121E000D1E0008BA
:100530001E00031E00001E02001E07001E0C001EEF
:1005400011001E17001E1C001E2100261E00211E69
:10055000001C1E00171E00111E000C1E00071E00AE
:10056000011E1E02001E07001E0C001E11001E1799
:10057000001E1C001E2100261E00211E001C1E0045
:10058000171E00111E000C1E00071E00021E000098
:100590001E02001E07001E0C001E11001E17001E6A
:1005A0001C001E2100261E00211E001C1E00171EFE
:1005B00000111E000C1E00071E00021E1E03001E5E
:1005C00007001E0C001E11001E17001E1C001E211D
:1005D00000261E00211E001C1E00171E00111E00FA
:1005E0000C1E00071E00021E00001E01001E070058
:1005F0001E0C001E11001E16001E1B001E20001ED9
:100600002500211E001C1E00171E00121E000D1EBC
:1006100000081E00031E1E03001E08001E0D001E03
:1006200012001E17001E1C001E2100251E00211E88
:10063000001C1E00171E00111E000C1E00071E00CD
:10064000021E00001E01001E07001E0C001E1100ED
:100650001E16001E1B001E20001E2500221E001D4F
:100660001E00181E00131E000E1E00081E00031E92
:100670001E04001E08001E0E001E13001E18001E81
:100680001C001E2100251E00201E001B1E00171E20
:1006900000111E000C1E00071E00021E00001E019D
:1006A000001E07001E0C001E11001E16001E1A0060
:1006B0001E1F001E2500221E001D1E00181E0013F6
:1006C0001E000E1E00091E00041E1E05001E09004D
:1006D0001E0E001E13001E18001E1D001E220025E7
:1006E0001E00201E001B1E00161E00111E000C1EE8
:1006F00000071E00021E00001E01001E07001E0C47
:10070000001E11001E15001E1A001E1F001E2400D0
:10071000231E001E1E00181E00141E000F1E000ABD
:100720001E00051E1E05001E0A001E0F001E1300DF
:100730001E18001E1E001E2200251E00201E001B6B
:100740001E00161E00111E000C1E00071E00021EB9
:1007500000001E01001E07001E0C001E10001E15CA
:10076000001E1A001E1F001E2400231E001E1E0055
:10077000191E00141E00101E000A1E00051E1E0673
:10078000001E0A001E0F001E14001E19001E1E006F
:100790001E2300241E00201E001A1E00161E00111B
:1007A0001E000C1E00071E00021E00001E01001E7F
:1007B00007001E0B001E10001E15001E1A001E1F33
:1007C000001E2300231E001E1E001A1E00151E0000
:1007D000101E000B1E00061E1E07001E0B001E1022
:1007E000001E15001E1A001E1E001E2300241E00DF
:1007F0001F1E001A1E00151E00111E000C1E0007F1
:100800001E00021E00001E01001E07001E0B001E1F
:1008100010001E15001E1A001E1E001E2300241E9E
:10082000001F1E001A1E00151E00111E000C1E00C7
:10083000071E1E07001E0C001E10001E15001E1AAB
:10084000001E1F001E2300231E001F1E001A1E0074
:10085000151E00111E000C1E00071E00021E0000C7
:100860001E01001E07001E0B001E10001E15001E9C
:1008700019001E1E001E2300241E001F1E001A1E2B
:1008800000161E00111E000C1E00071E1E08001E72
:100890000C001E11001E16001E1A001E1F001E2432
:1008A00000231E001E1E001A1E00151E00101E0032
:1008B0000C1E00071E00021E00001E01001E070085
:1008C0001E0B001E10001E15001E19001E1E001E0D
:1008D0002300251E001F1E001B1E00171E00111ED8
:1008E000000D1E00081E1E08001E0D001E11001E19
:1008F00016001E1B001E20001E2400231E001E1EAC
:10090000001A1E00151E00101E000C1E00071E00FF
:10091000021E00001E01001E06001E0B001E10001D
:100920001E14001E19001E1E001E2200251E00207F
:100930001E001C1E00171E00121E000E1E00081EA8
:100940001E09001E0E001E12001E17001E1B001E98
:1009500020001E2500231E001E1E00191E00151E4D
:1009600000101E000C1E00071E00021E00001E01CB
:10097000001E06001E0B001E10001E14001E180094
:100980001E1E001E2200251E00211E001C1E001718
:100990001E00131E000E1E00091E1E0A001E0E0061
:1009A0001E13001E17001E1C001E20001E25002204
:1009B0001E001E1E00191E00151E00101E000B1E1C
:1009C00000071E00021E00001E01001E06001E0A77
:1009D000001E10001E14001E18001E1D001E210007
:1009E000261E00211E001C1E00181E00131E000FD4
:1009F0001E000A1E1E0A001E0F001E13001E1800F5
:100A00001E1C001E21001E2500221E001E1E001995
:100A10001E00141E000F1E000B1E00071E00021EEB
:100A200000001E01001E06001E0A001E0F001E13FD
:100A3000001E18001E1D001E2100261E00211E0083
:100A40001D1E00181E00141E00101E000A1E1E0B84
:100A5000001E0F001E14001E18001E1D001E210087
:100A6000261E00211E001D1E00181E00141E000F51
:100A70001E000B1E00071E00021E00001E01001EAD
:100A800006001E0A001E0F001E13001E18001E1C6A
:100A9000001E21001E2500221E001E1E00191E0021
:100AA000151E00101E000B1E1E0C001E0F001E1433
:100AB000001E18001E1D001E2100261E00211E0003
:100AC0001D1E00181E00141E000F1E000B1E000726
:100AD0001E00021E00001E01001E06001E0A001E4F
:100AE0000F001E13001E18001E1C001E21001E25D4
:100AF00000221E001E1E00191E00151E00101E00E2
:100B00000C1E1E0C001E10001E15001E19001E1EBD
:100B1000001E2200251E00211E001C1E00181E00A3
:100B2000141E000F1E000B1E00071E00021E0000F8
:100B30001E01001E06001E0A001E0F001E13001ECE
:100B400017001E1C001E20001E2500231E001E1E56
:100B5000001A1E00151E00111E000C1E1E0D001E88
:100B600011001E15001E1A001E1E001E2300251E49
:100B700000211E001C1E00181E00131E000F1E0068
:100B80000B1E00071E00021E00001E01001E0600B4
:100B90001E0A001E0E001E13001E17001E1C001E43
:100BA00020001E2500231E001F1E001A1E00161EF8
:100BB00000111E000D1E1E0E001E11001E16001E2E
:100BC0001A001E1F001E2300251E00201E001C1ED2
:100BD00000181E00131E000F1E000A1E00071E0034
:100BE000021E00001E01001E06001E0A001E0E004E
:100BF0001E13001E17001E1B001E1F001E240023B4
:100C00001E001F1E001B1E00171E00121E000E1EBF
:100C10001E0E001E12001E17001E1B001E1F001EAF
:100C20002300241E00201E001C1E00171E00131E81
:100C3000000F1E000A1E00071E00021E00001E01FB
:100C4000001E06001E0A001E0E001E13001E1700C6
:100C50001E1B001E1F001E2300241E001F1E001C42
:100C60001E00171E00131E000E1E1E0F001E130076
:100C70001E17001E1B001E20001E2400241E002024
:100C80001E001C1E00171E00131E000F1E000A1E51
:100C900000061E00021E00001E01001E05001E0AA6
:100CA000001E0E001E12001E17001E1B001E1F003D
:100CB0001E2300251E00201E001C1E00181E0013EF
:100CC0001E000F1E1E0F001E13001E18001E1C000B
:100CD0001E20001E2400231E00201E001B1E0017C5
:100CE0001E00131E000E1E000A1E00061E00021E1D
:100CF00000001E01001E05001E0A001E0E001E122E
:100D0000001E17001E1A001E1F001E2300251E00B5
:100D1000211E001C1E00181E00141E00101E1E1096
:100D2000001E14001E18001E1C001E20001E2500A0
:100D3000231E001F1E001B1E00171E00131E000E88
:100D40001E000A1E00061E00021E00001E01001EDC
:100D500005001E0A001E0E001E12001E16001E1A9E
:100D6000001E1E001E2300251E00211E001D1E0049
:100D7000181E00151E00101E1E11001E15001E1844
:100D8000001E1D001E21001E2500231E001F1E0028
:100D90001A1E00171E00121E000E1E000A1E00065C
:100DA0001E00021E00001E01001E05001E0A001E7D
:100DB0000E001E11001E16001E1A001E1E001E220E
:100DC00000261E00211E001E1E00191E00151E00FA
:100DD000111E1E11001E15001E19001E1E001E21D0
:100DE000001E2500221E001E1E001A1E00161E00D8
:100DF000121E000E1E000A1E00061E00021E00002B
:100E00001E01001E05001E09001E0E001E11001E00
:100E100015001E1A001E1E001E2100261E00221E86
:100E2000001E1E001A1E00161E00111E1E12001E9D
:100E300016001E1A001E1E001E2200261E00221E64
:100E4000001E1E001A1E00161E00121E000E1E009E
:100E50000A1E00061E00021E00001E01001E0500E4
:100E60001E09001E0D001E11001E15001E19001E79
:100E70001E001E21001E2500231E001E1E001A1E1D
:100E800000171E00121E1E13001E17001E1A001E41
:100E90001E001E2200251E00211E001E1E001A1EFE
:100EA00000161E00111E000E1E000A1E00061E0067
:100EB000021E00001E01001E05001E09001E0D007E
:100EC0001E11001E15001E19001E1D001E21001EF1
:100ED0002500231E001F1E001B1E00171E00131ED0
:100EE0001E13001E17001E1B001E1F001E230025C0
:100EF0001E00211E001E1E00191E00151E00111EC0
:100F0000000E1E000A1E00061E00021E00001E012A
:100F1000001E05001E09001E0D001E11001E1500FA
:100F20001E18001E1D001E21001E2500231E001F6E
:100F30001E001C1E00181E00131E1E14001E18008A
:100F40001E1C001E20001E2300251E00211E001D49
:100F50001E00191E00151E00111E000E1E000A1E86
:100F600000061E00021E00001E01001E05001E09D4
:100F7000001E0D001E11001E15001E18001E1C0074
:100F80001E20001E2400241E00201E001C1E00180F
:100F90001E00141E1E15001E18001E1C001E200020
:100FA0001E2400241E00201E001C1E00181E0015FA
:100FB0001E00111E000D1E00091E00051E00011E50
:100FC00000001E01001E05001E09001E0D001E115E
:100FD000001E15001E18001E1C001E20001E2400EE
:100FE000241E00201E001C1E00181E00151E1E15AB
:100FF000001E18001E1C001E20001E2400241E00BF
:10100000201E001C1E00181E00151E00111E000DC3
:101010001E00091E00051E00011E00001E01001E0C
:1010200005001E08001E0C001E10001E14001E18D5
:10103000001E1C001E1F001E2300251E00211E0076
:101040001D1E00191E00151E1E16001E19001E1D55
:10105000001E21001E2500231E00201E001C1E0055
:10106000181E00151E00111E000D1E00091E000591
:101070001E00011E00001E01001E05001E08001EAD
:101080000C001E10001E14001E18001E1B001E1F48
:10109000001E2300251E00211E001E1E001A1E0019
:1010A000161E1E17001E1A001E1E001E21001E25E1
:1010B00000231E00201E001C1E00181E00141E000F
:1010C000111E000D1E00091E00051E00011E00005D
:1010D0001E01001E05001E08001E0C001E10001E32
:1010E00013001E17001E1B001E1F001E2300261EBD
:1010F00000221E001E1E001A1E00171E1E17001EB4
:101100001A001E1E001E22001E2500231E001F1E88
:10111000001B1E00181E00141E00101E000D1E00D5
:10112000091E00051E00011E00001E01001E050014
:101130001E08001E0C001E10001E13001E17001EAD
:101140001A001E1E001E2200261E00231E001F1E47
:10115000001B1E00171E1E18001E1B001E1F001E57
:101160002200261E00221E001F1E001B1E00171E2E
:1011700000141E00101E000C1E00091E00051E009B
:10118000011E00001E01001E05001E08001E0C00AE
:101190001E10001E13001E17001E1A001E1E001E29
:1011A00021001E2500231E001F1E001C1E00181EED
:1011B0001E18001E1C001E20001E2300251E0022DB
:1011C0001E001E1E001A1E00171E00131E00101EF9
:1011D000000C1E00081E00051E00011E00001E015E
:1011E000001E05001E08001E0C001E10001E13002D
:1011F0001E17001E1A001E1E001E21001E250023A1
:101200001E00201E001C1E00181E1E19001E1C00A1
:101210001E20001E2300251E00211E001E1E001A77
:101220001E00171E00131E000F1E000C1E00081EBD
:1012300000051E00011E00001E01001E05001E0804
:10124000001E0C001E0F001E13001E16001E1A00AA
:101250001E1D001E21001E2400241E00211E001D34
:101260001E00191E1E1A001E1D001E20001E240036
:10127000251E00211E001E1E001A1E00171E001330
:101280001E000F1E000C1E00081E00051E00011E81
:1012900000001E01001E05001E08001E0C001E0F8F
:1012A000001E12001E16001E19001E1D001E20002A
:1012B0001E2400251E00211E001E1E001A1E1E1ABE
:1012C000001E1E001E21001E2500241E00211E00DF
:1012D0001D1E001A1E00161E00131E000F1E000CFD
:1012E0001E00081E00051E00011E00001E01001E3B
:1012F00005001E08001E0B001E0F001E12001E150A
:10130000001E19001E1C001E20001E2300251E00AA
:10131000211E001E1E001A1E1E1B001E1E001E2166
:10132000001E2500231E00201E001D1E00191E0089
:10133000161E00131E000F1E000C1E00081E0005C6
:101340001E00011E00001E01001E04001E08001EDB
:101350000B001E0E001E12001E15001E18001E1C83
:10136000001E1F001E2300251E00221E001F1E003F
:101370001B1E1E1C001E1F001E22001E2500231EF9
:1013800000201E001C1E00191E00161E00121E004A
:101390000F1E000C1E00081E00051E00011E00008E
:1013A0001E01001E04001E08001E0B001E0E001E63
:1013B00011001E15001E18001E1C001E1F001E23FB
:1013C00000261E00231E001F1E001C1E1E1C001EC9
:1013D00020001E2300261E00231E00201E001C1EAF
:1013E00000181E00151E00121E000F1E000C1E000D
:1013F000081E00051E00011E00001E01001E040044
:101400001E07001E0B001E0E001E11001E15001EE2
:1014100018001E1B001E1F001E22001E2500231E7A
:1014200000201E001C1E1E1D001E20001E23002565
:101430001E00221E001F1E001C1E00181E00151E6E
:1014400000121E000E1E000B1E00081E00051E00CE
:10145000011E00001E01001E04001E07001E0A00DF
:101460001E0E001E11001E15001E18001E1B001E61
:101470001E001E21001E2500241E00211E001D1E10
:101480001E1E001E21001E2400251E00211E001EFF
:101490001E001B1E00181E00151E00111E000E1E31
:1014A000000B1E00081E00051E00011E00001E018C
:1014B000001E04001E07001E0A001E0E001E110062
:1014C0001E14001E17001E1A001E1E001E21001EE4
:1014D0002400251E00211E001E1E1E1E001E2100AF
:1014E0001E2400251E00211E001E1E001B1E0018AB
:1014F0001E00151E00111E000E1E000B1E00081EF1
:1015000000051E00011E00001E01001E04001E0733
:10151000001E0A001E0E001E11001E14001E1700E1
:101520001E1A001E1E001E21001E2400251E002162
:101530001E001E1E1E1F001E21001E2500241E0050
:10154000211E001E1E001A1E00171E00141E001170
:101550001E000E1E000B1E00081E00051E00011EB0
:1015600000001E01001E04001E07001E0A001E0EC1
:10157000001E10001E13001E17001E1A001E1D0064
:101580001E20001E2300251E00221E001F1E1E20DE
:10159000001E22001E2500231E00201E001D1E000E
:1015A0001A1E00171E00141E00111E000E1E000A37
:1015B0001E00081E00051E00011E00001E01001E68
:1015C00004001E07001E0A001E0D001E10001E1340
:1015D000001E17001E1A001E1C001E1F001E2300E6
:1015E000261E00231E001F1E1E20001E2300261E76
:1015F00000231E00201E001D1E001A1E00171E00C4
:10160000131E00111E000E1E000A1E00071E0005FC
:101610001E00011E00001E01001E04001E07001E09
:101620000A001E0D001E10001E13001E16001E19BB
:10163000001E1C001E1F001E22001E2500231E006F
:10164000201E1E21001E2300251E00221E00201E1B
:10165000001C1E00191E00171E00131E00101E0085
:101660000E1E000A1E00071E00051E00011E0000BF
:101670001E01001E04001E07001E0A001E0D001E93
:1016800010001E13001E16001E18001E1C001E1F38
:10169000001E21001E2500241E00211E1E21001EEA
:1016A0002400251E00221E001F1E001C1E00191EE5
:1016B00000161E00131E00101E000D1E000A1E0044
:1016C000071E00041E00011E00001E01001E030074
:1016D0001E07001E0A001E0C001E10001E13001E16
:1016E00015001E18001E1B001E1E001E21001E24B9
:1016F00000251E00211E1E22001E2500241E002182
:101700001E001E1E001C1E00181E00161E00131EAA
:1017100000101E000D1E000A1E00071E00041E0001
:10172000011E00001E01001E03001E07001E09000E
:101730001E0C001E10001E12001E15001E18001E9A
:101740001B001E1E001E21001E2300251E00221E3F
:101750001E23001E2500241E00211E001E1E001B2D
:101760001E00181E00151E00131E000F1E000D1E69
:10177000000A1E00071E00041E00011E00001E01BC
:10178000001E03001E07001E09001E0C001E0F0095
:101790001E12001E15001E18001E1A001E1E001E1E
:1017A00020001E2300261E00231E1E2300261E00CE
:1017B000231E00201E001E1E001A1E00181E0015EB
:1017C0001E00121E000F1E000C1E000A1E00071E27
:1017D00000041E00011E00001E01001E03001E0763
:1017E000001E09001E0C001E0F001E11001E150019
:1017F0001E17001E1A001E1D001E1F001E23001EA5
:101800002500231E1E2400251E00231E00201E006E
:101810001D1E001A1E00171E00151E00121E000FAE
:101820001E000C1E000A1E00071E00041E00011EE2
:1018300000001E01001E03001E06001E09001E0CF3
:10184000001E0E001E11001E14001E17001E1A009E
:101850001E1C001E1F001E22001E2500241E1E2509
:1018600000251E00221E00201E001C1E001A1E0045
:10187000171E00151E00111E000F1E000C1E000971
:101880001E00071E00041E00011E00001E01001E97
:1018900003001E06001E08001E0C001E0E001E1176
:1018A000001E14001E17001E19001E1C001E1F0023
:1018B0001E21001E2400251E1E2500241E00211EA0
:1018C000001F1E001C1E00191E00171E00141E0003
:1018D000111E000F1E000C1E00091E00071E000432
:1018E0001E00011E00001E01001E03001E06001E39
:1018F00008001E0B001E0E001E11001E13001E16F7
:10190000001E18001E1C001E1E001E21001E2300AB
:10191000251E261E00231E00211E001E1E001C1E4A
:1019200000191E00171E00141E00111E000E1E00BE
:101930000C1E00091E00071E00041E00011E0000F0
:101940001E01001E03001E06001E08001E0B001EC6
:101950000E001E10001E13001E16001E18001E1B77
:10196000001E1E001E20001E2300261E251E002312
:101970001E00201E001E1E001B1E00181E00161E2C
:1019800000131E00111E000E1E000C1E00091E007A
:10199000071E00041E00011E00001E01001E0300A1
:1019A0001E06001E08001E0B001E0E001E10001E4C
:1019B00013001E15001E18001E1A001E1D001E1FFB
:1019C000001E22001E25251E00221E00201E001DB6
:1019D0001E001A1E00181E00151E00131E00101EE9
:1019E000000E1E000B1E00081E00061E00031E0037
:1019F000011E00001E01001E03001E06001E08003E
:101A00001E0B001E0E001E10001E13001E15001ED1
:101A100018001E1A001E1D001E1F001E22001E257B
:101A2000241E00221E00201E001D1E001A1E00186B
:101A30001E00151E00131E00101E000E1E000B1EA1
:101A400000081E00061E00031E00011E00001E00EE
:101A5000001E03001E05001E08001E0A001E0D00C9
:101A60001E10001E12001E15001E17001E1A001E5A
:101A70001C001E1F001E21001E24231E00211E000C
:101A80001F1E001C1E001A1E00171E00151E00122D
:101A90001E00101E000E1E000B1E00081E00061E5B
:101AA00000031E00011E00001E00001E03001E0594
:101AB000001E08001E0A001E0D001E10001E110050
:101AC0001E14001E17001E19001E1C001E1E001EE4
:101AD00021001E23231E00211E001E1E001C1E00AE
:101AE000191E00171E00151E00121E000F1E000DED
:101AF0001E000B1E00081E00061E00031E00011E15
:101B000000001E00001E03001E05001E08001E0A25
:101B1000001E0C001E0F001E11001E14001E1700D8
:101B20001E18001E1B001E1E001E20001E23221E4B
:101B300000201E001E1E001B1E00191E00171E0086
:101B4000141E00111E000F1E000D1E000A1E0008AC
:101B50001E00061E00031E00011E00001E00001EC7
:101B600003001E05001E08001E0A001E0C001E0FAA
:101B7000001E11001E13001E16001E18001E1A0063
:101B80001E1D001E1F001E22211E00201E001D1EE5
:101B9000001B1E00181E00161E00141E00111E0041
:101BA0000F1E000D1E000A1E00081E00061E000368
:101BB0001E00011E00001E00001E03001E05001E68
:101BC00007001E0A001E0C001E0E001E11001E1330
:101BD000001E15001E18001E1A001E1C001E1F00ED
:101BE0001E21211E001F1E001C1E001A1E00181E92
:101BF00000161E00131E00111E000F1E000C1E00FA
:101C00000A1E00081E00051E00031E00011E000023
:101C10001E00001E03001E05001E07001E0A001EF7
:101C20000C001E0E001E10001E13001E15001E17B5
:101C3000001E1A001E1C001E1E001E21201E001E5B
:101C40001E001C1E001A1E00171E00151E00131E6B
:101C500000111E000E1E000C1E000A1E00081E00B1
:101C6000051E00031E00011E00001E00001E0300D2
:101C70001E05001E07001E09001E0C001E0E001E81
:101C800010001E12001E15001E17001E19001E1B3C
:101C9000001E1E001E20201E001E1E001C1E0019FD
:101CA0001E00171E00151E00131E00101E000E1E23
:101CB000000C1E000A1E00081E00051E00031E0068
:101CC000011E00001E00001E03001E05001E07006E
:101CD0001E09001E0B001E0E001E10001E12001E0C
:101CE00014001E17001E18001E1B001E1D001E1FC4
:101CF0001F1E001D1E001B1E00181E00171E0015B3
:101D00001E00121E00101E000E1E000C1E000A1ED9
:101D100000071E00051E00031E00011E00001E001D
:101D2000001E03001E05001E07001E09001E0B00FA
:101D30001E0D001E10001E11001E14001E16001E97
:101D400018001E1A001E1C001E1F1E1E001C1E0056
:101D50001A1E00181E00161E00141E00121E000F70
:101D60001E000E1E000C1E00091E00071E00051E90
:101D700000031E00011E00001E00001E02001E05C2
:101D8000001E07001E08001E0B001E0D001E0F0087
:101D90001E11001E13001E15001E18001E1A001E24
:101DA0001C001E1E1E1E001C1E001A1E00181E00F7
:101DB000161E00131E00111E000F1E000E1E000B2B
:101DC0001E00091E00071E00051E00031E00011E46
:101DD00000001E00001E02001E05001E07001E0857
:101DE000001E0A001E0D001E0F001E11001E130013
:101DF0001E15001E17001E19001E1B001E1E1D1E94
:101E0000001B1E00191E00171E00151E00131E00C9
:101E1000111E000F1E000D1E000B1E00091E0007E4
:101E20001E00051E00031E00011E00001E00001EF5
:101E300002001E04001E07001E08001E0A001E0CE1
:101E4000001E0E001E10001E13001E15001E17009F
:101E50001E18001E1A001E1D1C1E001A1E00181E31
:101E600000171E00151E00131E00111E000F1E007D
:101E70000D1E000B1E00081E00071E00051E00039D
:101E80001E00011E00001E00001E02001E04001E97
:101E900006001E08001E0A001E0C001E0E001E106A
:101EA000001E12001E14001E16001E18001E1A002E
:101EB0001E1C1C1E001A1E00181E00161E00141EDA
:101EC00000121E00101E000E1E000C1E000A1E0036
:101ED000081E00071E00051E00031E00011E000054
:101EE0001E00001E02001E04001E06001E08001E2A
:101EF0000A001E0C001E0E001E10001E11001E13F4
:101F0000001E15001E17001E19001E1C1B1E001AA5
:101F10001E00181E00161E00141E00121E00101EA9
:101F2000000E1E000C1E000A1E00081E00071E00E8
:101F3000051E00031E00011E00001E00001E020000
:101F40001E04001E06001E08001E0A001E0C001EB5
:101F50000E001E10001E11001E13001E15001E177D
:101F6000001E19001E1B1A1E00191E00171E001548
:101F70001E00131E00111E000F1E000E1E000C1E60
:101F8000000A1E00081E00071E00051E00031E009A
:101F9000011E00001E00001E02001E04001E06009E
:101FA0001E08001E09001E0B001E0D001E0F001E45
:101FB00011001E13001E15001E17001E18001E1A09
:101FC0001A1E00181E00171E00151E00131E0011F9
:101FD0001E000F1E000E1E000C1E000A1E00081E12
:101FE00000061E00051E00031E00011E00001E004C
:101FF000001E02001E04001E05001E07001E090030
:102000001E0B001E0D001E0F001E10001E12001ED3
:1020100014001E16001E18001E1A191E00181E009D
:10202000161E00141E00121E00111E000F1E000DB1
:102030001E000B1E000A1E00081E00061E00041EC5
:1020400000031E00011E00001E00001E02001E03F1
:10205000001E05001E07001E09001E0A001E0C00BF
:102060001E0E001E10001E11001E13001E15001E65
:1020700017001E19181E00171E00151E00131E0043
:10208000121E00101E000E1E000D1E000B1E000969
:102090001E00081E00061E00041E00031E00011E76
:1020A00000001E00001E02001E03001E05001E0789
:1020B000001E08001E0A001E0C001E0E001E10004E
:1020C0001E11001E13001E15001E17001E18181EDC
:1020D00000171E00151E00131E00111E000F1E000B
:1020E0000E1E000C1E000B1E00091E00071E00061F
:1020F0001E00041E00021E00011E00001E00001E25
:1021000001001E03001E05001E07001E08001E0A17
:10211000001E0C001E0E001E0F001E11001E1300DC
:102120001E14001E16001E18171E00161E00141E78
:1021300000131E00111E000F1E000E1E000C1E00BC
:102140000A1E00091E00071E00051E00041E0002D4
:102150001E00011E00001E00001E01001E03001EC6
:1021600005001E07001E08001E0A001E0C001E0DA2
:10217000001E0F001E10001E12001E13001E150070
:102180001E17171E00151E00141E00121E00111E21
:10219000000F1E000E1E000C1E000A1E00081E006E
:1021A000071E00051E00041E00021E00011E000086
:1021B0001E00001E01001E03001E05001E07001E5B
:1021C00008001E0A001E0B001E0D001E0E001E1031
:1021D000001E11001E13001E15001E17161E0015EE
:1021E0001E00131E00111E00101E000E1E000D1EEC
:1021F000000C1E000A1E00081E00071E00051E001F
:10220000041E00021E00011E00001E00001E010030
:102210001E03001E05001E06001E08001E09001EEB
:102220000B001E0C001E0E001E10001E11001E13BF
:10223000001E14001E16151E00141E00131E001191
:102240001E000F1E000E1E000C1E000B1E000A1E9C
:1022500000081E00071E00051E00031E00021E00CF
:10226000011E00001E00001E01001E03001E0500CE
:102270001E06001E07001E09001E0A001E0C001E7E
:102280000E001E0F001E10001E12001E13001E1551
:10229000151E00131E00121E00111E000F1E000E40
:1022A0001E000C1E000B1E00091E00081E00071E4B
:1022B00000051E00031E00021E00011E00001E007D
:1022C000001E01001E03001E04001E06001E070063
:1022D0001E08001E0A001E0C001E0D001E0E001E11
:1022E00010001E11001E13001E15141E00131E00E8
:1022F000111E00101E000F1E000D1E000C1E000AF5
:102300001E00091E00081E00061E00051E00031EFA
:1023100000021E00011E00001E00001E01001E0320
:10232000001E04001E05001E07001E08001E0A00F5
:102330001E0B001E0C001E0E001E10001E11001EA3
:1023400012001E14131E00121E00111E000F1E008C
:102350000E1E000D1E000C1E000A1E00081E0007A7
:102360001E00061E00051E00031E00021E00011EA8
:1023700000001E00001E01001E03001E04001E05BA
:10238000001E07001E08001E0A001E0B001E0C0087
:102390001E0E001E0F001E10001E11001E13131E25
:1023A00000111E00101E000F1E000E1E000C1E004D
:1023B0000B1E000A1E00081E00071E00061E000558
:1023C0001E00031E00021E00011E00001E00001E53
:1023D00001001E03001E04001E05001E07001E084B
:1023E000001E09001E0A001E0C001E0D001E0E001D
:1023F0001E10001E11001E13121E00111E000F1EC3
:10240000000E1E000D1E000C1E000A1E00091E00FC
:10241000081E00071E00051E00041E00031E00010A
:102420001E00001E00001E00001E01001E03001EF4
:1024300004001E05001E07001E08001E09001E0ADB
:10244000001E0C001E0D001E0E001E10001E1100AE
:102450001E12111E00111E000F1E000E1E000D1E6A
:10246000000C1E000A1E00091E00081E00071E00A8
:10247000051E00041E00031E00011E00001E0000B9
:102480001E00001E01001E02001E03001E05001E8D
:1024900006001E07001E08001E0A001E0B001E0C70
:1024A000001E0E001E0F001E10001E11111E001037
:1024B0001E000F1E000E1E000C1E000B1E000A1E2A
:1024C00000081E00081E00071E00051E00041E0056
:1024D000031E00011E00001E00001E00001E010061
:1024E0001E02001E03001E05001E06001E07001E21
:1024F00008001E09001E0A001E0C001E0D001E0E04
:10250000001E10001E11101E000F1E000E1E000DDA
:102510001E000C1E000B1E000A1E00081E00071ED7
:1025200000061E00051E00041E00031E00011E0002
:10253000001E00001E00001E01001E02001E0300FF
:102540001E05001E05001E07001E08001E09001EB5
:102550000A001E0B001E0C001E0E001E0F001E1097
:102560000F1E000F1E000E1E000C1E000C1E000A87
:102570001E00091E00081E00071E00061E00051E84
:1025800000041E00031E00011E00001E00001E00AD
:10259000001E01001E02001E03001E04001E050096
:1025A0001E07001E07001E08001E0A001E0B001E4C
:1025B0000C001E0D001E0E001E100F1E000E1E0031
:1025C0000D1E000C1E000B1E000A1E00091E000836
:1025D0001E00071E00061E00051E00031E00031E2F
:1025E00000011E00001E00001E00001E01001E0251
:1025F000001E03001E04001E05001E06001E07002C
:102600001E08001E09001E0A001E0C001E0C001EE3
:102610000E001E0F0E1E000E1E000C1E000C1E00D3
:102620000A1E000A1E00081E00071E00071E0005E5
:102630001E00051E00031E00021E00011E00001EDB
:1026400000001E00001E01001E01001E03001E04EB
:10265000001E05001E06001E07001E08001E0900C1
:102660001E0A001E0B001E0C001E0D001E0E0E1E6C
:10267000000D1E000C1E000B1E000A1E00091E008D
:10268000081E00071E00061E00051E00041E000393
:102690001E00021E00011E00001E00001E00001E83
:1026A00001001E01001E03001E03001E05001E0582
:1026B000001E07001E07001E08001E09001E0A005B
:1026C0001E0B001E0C001E0E0D1E000C1E000C1E0C
:1026D000000A1E000A1E00081E00081E00071E0039
:1026E000061E00051E00041E00031E00021E00013F
:1026F0001E00001E00001E00001E01001E01001E24
:1027000003001E03001E04001E05001E06001E0717
:10271000001E08001E09001E0A001E0B001E0C00F1
:102720001E0D0C1E000C1E000B1E000A1E00091EB2
:1027300000081E00071E00071E00051E00051E00E3
:10274000041E00031E00021E00011E00001E0000E9
:102750001E00001E01001E01001E02001E03001EBE
:1027600004001E05001E06001E07001E08001E08AD
:10277000001E09001E0A001E0B001E0C0C1E000B82
:102780001E000A1E000A1E00081E00081E00071E6A
:1027900000061E00051E00051E00031E00031E008D
:1027A000021E00011E00001E00001E00001E000090
:1027B0001E01001E02001E03001E04001E05001E56
:1027C00005001E07001E07001E08001E09001E0A45
:1027D000001E0A001E0C0B1E000A1E000A1E000925
:1027E0001E00081E00071E00071E00061E00051E14
:1027F00000041E00031E00031E00021E00011E0036
:10280000001E00001E00001E00001E01001E02002F
:102810001E03001E03001E05001E05001E06001EEE
:1028200007001E08001E08001E09001E0A001E0BDD
:102830000A1E000A1E00091E00081E00081E0007CE
:102840001E00061E00051E00051E00041E00031EBD
:1028500000031E00011E00011E00001E00001E00DD
:10286000001E00001E01001E02001E03001E0300C9
:102870001E04001E05001E05001E07001E07001E88
:1028800008001E08001E09001E0A0A1E00091E007C
:10289000081E00081E00071E00071E00061E000579
:1028A0001E00051E00041E00031E00021E00011E65
:1028B00000011E00001E00001E00001E00001E0180
:1028C000001E01001E02001E03001E04001E050063
:1028D0001E05001E06001E07001E07001E08001E23
:1028E00008001E0A091E00081E00081E00071E0020
:1028F000071E00061E00051E00051E00041E000324
:102900001E00031E00021E00011E00011E00001E0C
:1029100000001E00001E00001E01001E01001E021D
:10292000001E03001E03001E04001E05001E0500FD
:102930001E06001E07001E07001E08001E09081EB6
:1029400000081E00081E00071E00071E00061E00CD
:10295000051E00051E00041E00031E00031E0002CB
:102960001E00011E00011E00001E00001E00001EB1
:1029700000001E01001E01001E02001E03001E03B7
:10298000001E04001E05001E05001E06001E070096
:102990001E07001E08001E08081E00081E00071E55
:1029A00000071E00061E00051E00051E00041E0076
:1029B000031E00031E00031E00021E00011E000174
:1029C0001E00001E00001E00001E00001E01001E52
:1029D00001001E02001E02001E03001E03001E0452
:1029E000001E05001E05001E06001E07001E070033
:1029F0001E08071E00071E00071E00061E00051EFB
:102A000000051E00051E00041E00031E00031E001C
:102A1000021E00011E00011E00011E00001E00001B
:102A20001E00001E00001E01001E01001E01001EEF
:102A300002001E03001E03001E04001E04001E05EB
:102A4000001E05001E06001E07001E07071E0007C9
:102A50001E00061E00051E00051E00051E00041EA9
:102A600000031E00031E00031E00021E00011E00C4
:102A7000011E00011E00001E00001E00001E0000BE
:102A80001E00001E01001E01001E02001E02001E8C
:102A900003001E03001E04001E04001E05001E0588
:102AA000001E06001E07061E00061E00051E00056D
:102AB0001E00051E00041E00031E00031E00031E50
:102AC00000021E00021E00011E00011E00011E0069
:102AD000001E00001E00001E00001E00001E01005F
:102AE0001E01001E01001E02001E03001E03001E28
:102AF00003001E04001E04001E05001E05001E0625
:102B0000051E00051E00051E00051E00041E000314
:102B10001E00031E00031E00031E00021E00011EF5
:102B200000011E00011E00001E00001E00001E000D
:102B3000001E00001E00001E01001E01001E0100FC
:102B40001E02001E02001E03001E03001E03001EC4
:102B500004001E04001E05001E05051E00051E00C3
:102B6000041E00041E00031E00031E00031E0003BB
:102B70001E00021E00021E00011E00011E00011E9A
:102B800000001E00001E00001E00001E00001E00AF
:102B9000001E00001E01001E01001E01001E02009A
:102BA0001E02001E03001E03001E03001E03001E63
:102BB00004001E05041E00041E00041E00031E0067
:102BC000031E00031E00031E00021E00021E000161
:102BD0001E00011E00011E00011E00001E00001E3E
:102BE00000001E00001E00001E00001E00001E014E
:102BF000001E01001E01001E01001E02001E020038
:102C00001E03001E03001E03001E03001E04031EFD
:102C100000031E00031E00031E00031E00021E0010
:102C2000021E00021E00011E00011E00011E000106
:102C30001E00011E00001E00001E00001E00001EDF
:102C400000001E00001E00001E00001E01001E01EC
:102C5000001E01001E01001E01001E02001E0200D7
:102C60001E03001E03001E03031E00031E00031E9E
:102C700000021E00021E00021E00011E00011E00B6
:102C8000011E00011E00011E00011E00001E0000AA
:102C90001E00001E00001E00001E00001E00001E80
:102CA00000001E00001E00001E01001E01001E018B
:102CB000001E01001E01001E01001E02001E020077
:102CC0001E03021E00021E00021E00021E00011E44
:102CD00000011E00011E00011E00011E00011E0059
:102CE000011E00001E00001E00001E00001E00004D
:102CF0001E00001E00001E00001E00001E00001E20
:102D000000001E00001E01001E01001E01001E0129
:102D1000001E01001E01001E01001E02011E000116
:102D20001E00011E00011E00011E00011E00011EEA
:102D300000011E00011E00011E00001E00001E00FA
:102D4000001E00001E00001E00001E00001E0000ED
:102D50001E00001E00001E00001E00001E00001EBF
:102D600000001E00001E00001E01001E01001E01CA
:102D7000001E01001E01011E00011E00011E0001B7
:102D80001E00011E00011E00011E00011E00001E8B
:102D900000001E00001E00001E00001E00001E009D
:102DA000001E00001E00001E00001E00001E00008D
:102DB0001E00001E00001E00001E00001E00001E5F
:102DC00000001E00001E00001E00001E00001E016C
:102DD000001E00001E00001E00001E00001E00005D
:102DE0001E00001E00001E00001E00001E00001E2F
:102DF00000001E00001E00001E00001E00001E003D
:102E0000001E00001E00001E00001E00001E00002C
:102E10001E00001E00001E00001E00001E00001EFE
:102E200000001E00001E00001E0011241FBECFEF78
:102E3000D8E0DEBFCDBF0E947F190C94181C0C9403
:102E400000008C0181E087B9C0E0D0E0C017D10755
:102E50003CF440E060E085E50E946D172196F6CFD6
:102E60002FEF86EB90E2215080409040E1F700C0C8
:102E70000000C0E0D0E0C017D1073CF445E560E0B9
:102E800080E00E946D172196F6CF2FEF86EB90E23F
:102E9000215080409040E1F700C00000D5CF81E094
:102EA00088B900C000C000C018B800C000C000C091
:102EB00000C000C000C000C00000089581E088B9D3
:102EC00000C000C000C000C000C000C000C018B8F2
:102ED00000C000C000C000C00895AF92BF92CF9262
:102EE000DF92EF92FF920F931F93CF93DF93C82E41
:102EF000E42EC8E0D0E000E810E0A62EB12CC80116
:102F00008A219B21892B19F00E945E1702C00E9422
:102F10004F1715950795219791F7C8E0D0E000E885
:102F200010E0D12CC8018C219D21892B19F00E9421
:102F30005E1702C00E944F1715950795219791F7CC
:102F4000C8E0D0E000E810E0F12CC8018E219F21FC
:102F5000892B19F00E945E1702C00E944F17159529
:102F60000795219791F7DF91CF911F910F91FF90D6
:102F7000EF90DF90CF90BF90AF9008952F923F9247
:102F80004F925F926F927F928F929F92AF92BF9279
:102F9000CF92DF92EF92FF920F931F93CF93DF9325
:102FA000CDB7DEB72A970FB6F894DEBF0FBECDBF00
:102FB000D82EC92EF7010130110501F13B0129017D
:102FC000461A570A842F90E0BC016D1971097E835F
:102FD0006D83852F90E09C012C19310938872F8350
:102FE00033961A861986E12CF12C80E090E020E0DF
:102FF00030E0580141E0A41AB10805C06083718334
:10300000828393833DC01C01240C351C4D815E815D
:103010004E0D5F1D5A8349834F81588569857A8596
:10302000460F571F5C834B832017310749F14F012F
:1030300053E0851A9108B5010E94EA1B660D771DC1
:10304000D4016D937C934F01B1E08B1A9108C701B5
:10305000B5010E94EA1B6D0DD4016C9389859A8598
:10306000B5010E94EA1B6C0D60832F5F3F4F3496C1
:103070004B815C815A874987E980FA80C101C3CFBF
:103080002A960FB6F894DEBF0FBECDBFDF91CF9169
:103090001F910F91FF90EF90DF90CF90BF90AF9076
:1030A0009F908F907F906F905F904F903F902F9068
:1030B00008952F923F924F925F926F927F928F92DC
:1030C0009F92AF92BF92CF92DF92EF92FF920F93B7
:1030D0001F93CF93DF9300D000D0CDB7DEB7FC01B4
:1030E000B2803380B11004C0232C3B823C82C2C02A
:1030F000FC0100811181B8010836F1E01F0710F0D2
:103100006856714080E090E00E94EF1A2B013C016C
:10311000632D70E080E090E00E94EF1A20E030E044
:1031200048EC52E40E944E1A6B017C016B2D70E05A
:1031300080E090E00E94EF1A20E030E048EC52E49A
:103140000E944E1A4B015C0120E030E040E752E45F
:10315000C301B2010E944E1A2B013C010E94C01A09
:103160006A8370E080E090E00E94F11A9B01AC015C
:10317000C301B2010E94E1192B013C01A501940198
:1031800060E070E080E89FE30E94E1199B01AC01E0
:10319000C701B6010E947D1B20E030E040E053E40F
:1031A0000E947D1B0E94C01A262EA3019201C50118
:1031B000B4010E947D1B9B01AC0160E070E080E8DF
:1031C0009FE30E94E1199B01AC01C701B6010E9477
:1031D0007D1B20E030E040E053E40E947D1B0E9414
:1031E000C01A6983A301920160E070E080E89FE368
:1031F0000E94E1199B01AC01C501B4010E947D1B35
:103200009B01AC0160E070E080E89FE30E94E1195F
:103210009B01AC01C701B6010E947D1B20E030E09C
:1032200040E053E40E947D1B0E94C01A2A81822F35
:1032300090E087309105E8F4FC01EC5CFF4F0C94C2
:10324000FE1B2B826C83232C15C02B823C82298091
:1032500011C06B833C820EC03B8289818C830AC083
:103260003B822C82262E06C0E981EB832C82202E05
:1032700001C0212C622D7C818B810F900F900F90CB
:103280000F90DF91CF911F910F91FF90EF90DF9002
:10329000CF90BF90AF909F908F907F906F905F90F6
:1032A0004F903F902F900895CF92DF92EF92FF9230
:1032B0000F931F93CF93DF936A01EB017C0100E032
:1032C00010E00C151D0561F0C7010E9459186993A3
:1032D000799389930F5F1F4F84E0E80EF11CF1CFC3
:1032E000DF91CF911F910F91FF90EF90DF90CF90E2
:1032F0000895282F862F622F792F942F089581E02B
:1033000087B911E080E090E0C0E0D0E03DE1E32E3D
:10331000F12C0AE51130D9F40C9F60010D9FD00CFF
:103320001124A12CB12CF501EC0DFD1DEA58FF4F25
:103330004281618180810E946D1723E0A20EB11C41
:103340003AE5A316B10479F78EE190E023C01F3F60
:1033500009F5F701E81BF90B8EE1C82ED12CCF013E
:10336000880F991FE80FF91F0C9FC0010D9F900D4A
:103370001124E80FF91FEA58FF4F9280A180B08016
:10338000492D6A2D8B2D0E946D1741E0C41AD1087A
:10339000B9F7DACF2FE33DE043E021503040404021
:1033A000E1F700C00000C10FD11D17FDDA95C1384B
:1033B000D10511F41FEFCDCF209709F0ABCF11E06D
:1033C000ABCF5058BB27AA270E94F9190C94431B76
:1033D0000E94351B38F00E943C1B20F039F49F3FBF
:1033E00019F426F40C94321B0EF4E095E7FB0C94D0
:1033F0002C1BE92F0E94541B58F3BA17620773075E
:103400008407950720F079F4A6F50C94761B0EF44A
:10341000E0950B2EBA2FA02D0B01B90190010C01E4
:10342000CA01A0011124FF27591B99F0593F50F4FC
:10343000503E68F11A16F040A22F232F342F442754
:10344000585FF3CF469537952795A795F04053954C
:10345000C9F77EF41F16BA0B620B730B840BBAF01C
:103460009150A1F0FF0FBB1F661F771F881FC2F787
:103470000EC0BA0F621F731F841F48F4879577959B
:103480006795B795F7959E3F08F0B0CF9395880F55
:1034900008F09927EE0F9795879508950E94621A74
:1034A0000C94431B0E943C1B58F00E94351B40F0BB
:1034B00029F45F3F29F00C942C1B51110C94771BBD
:1034C0000C94321B0E94541B68F39923B1F35523CB
:1034D00091F3951B550BBB27AA2762177307840727
:1034E00038F09F5F5F4F220F331F441FAA1FA9F3BD
:1034F00035D00E2E3AF0E0E832D091505040E695AB
:10350000001CCAF72BD0FE2F29D0660F771F881F0B
:10351000BB1F261737074807AB07B0E809F0BB0BFE
:10352000802DBF01FF2793585F4F3AF09E3F510512
:1035300078F00C942C1B0C94771B5F3FE4F3983EBF
:10354000D4F3869577956795B795F7959F5FC9F7FB
:10355000880F911D9695879597F90895E1E0660F7C
:10356000771F881FBB1F621773078407BA0720F0F5
:10357000621B730B840BBA0BEE1F88F7E09508955E
:103580000E945C1B88F09F5798F0B92F9927B7517C
:10359000B0F0E1F0660F771F881F991F1AF0BA95F7
:1035A000C9F714C0B13091F00E94761BB1E00895C4
:1035B0000C94761B672F782F8827B85F39F0B93FB6
:1035C000CCF3869577956795B395D9F73EF49095AA
:1035D0008095709561957F4F8F4F9F4F0895E89428
:1035E00009C097FB3EF490958095709561957F4F4B
:1035F0008F4F9F4F9923A9F0F92F96E9BB279395F9
:10360000F695879577956795B795F111F8CFFAF408
:10361000BB0F11F460FF1BC06F5F7F4F8F4F9F4F39
:1036200016C0882311F096E911C0772321F09EE897
:10363000872F762F05C0662371F096E8862F70E0FD
:1036400060E02AF09A95660F771F881FDAF7880FD7
:103650009695879597F9089597F99F6780E870E0A8
:1036600060E008959FEF80EC089500240A941616F8
:10367000170618060906089500240A941216130660
:10368000140605060895092E0394000C11F48823EE
:1036900052F0BB0F40F4BF2B11F460FF04C06F5F0A
:1036A0007F4F8F4F9F4F089557FD9058440F551FE0
:1036B00059F05F3F71F04795880F97FB991F61F0B4
:1036C0009F3F79F087950895121613061406551F2B
:1036D000F2CF4695F1DF08C0161617061806991F97
:1036E000F1CF86957105610508940895E894BB278C
:1036F00066277727CB0197F908950E94901B0C94B9
:10370000431B0E94351B38F00E943C1B20F0952380
:1037100011F00C942C1B0C94321B11240C94771B6D
:103720000E94541B70F3959FC1F3950F50E0551FF5
:10373000629FF001729FBB27F00DB11D639FAA2706
:10374000F00DB11DAA1F649F6627B00DA11D661F55
:10375000829F2227B00DA11D621F739FB00DA11D76
:10376000621F839FA00D611D221F749F3327A00D30
:10377000611D231F849F600D211D822F762F6A2FCC
:1037800011249F5750409AF0F1F088234AF0EE0F31
:10379000FF1FBB1F661F771F881F91505040A9F75E
:1037A0009E3F510580F00C942C1B0C94771B5F3FBF
:1037B000E4F3983ED4F3869577956795B795F7959A
:1037C000E7959F5FC1F7FE2B880F911D9695879512
:1037D00097F9089597FB072E16F4009407D077FD0C
:1037E00009D00E94041C07FC05D03EF490958195F9
:1037F0009F4F0895709561957F4F0895EE0FFF1FBD
:103800000590F491E02D0994AA1BBB1B51E107C060
:10381000AA1FBB1FA617B70710F0A61BB70B881F60
:10382000991F5A95A9F780959095BC01CD010895EF
:04383000F894FFCF3A
:00000001FF
